:020000040000FA
:020000000528D1
:08000800C02803138316083021
:10001000810002308E008312850107309F00831615
:100020000C1083120130900083161030850083126B
:1000300040308500831686018312FF3086008B12C4
:100040000B178B1785152F142F0803192928A520A6
:10005000AF01051A24281E30B720051A24288B1258
:100060008316FF30860083120030A0000130A1000B
:10007000A301A401AB012008403885000000000066
:10008000000006092106A304712020088620A20092
:1000900006092206A404FA30B720A00A0310A10D15
:1000A000031C3B28483085008316860183122408F0
:1000B000031D5D28860005136528230886002B088C
:1000C000483885002B08031D6728902068289E204B
:1000D000A8010030A9003230AA00103081008B1630
:1000E00024280609031D76282B148528A600031052
:1000F000A60C031C7828A60803198028AB148528B1
:1001000006092106031985282B1508000F398207D7
:100110000434203401340834103402344034803440
:100120000030AC000330AD001930AE00AA2800301A
:10013000AC000530AD001930AE00AA280030AC008C
:100140000730AD004130AE00AA2897201E30B720FE
:100150009020080085172D08A700A70BAD28851350
:100160002D08A700A70BB228AE0BAA280800A500EF
:100170000000BA28BB28BC28BD28A50BB828080059
:10018000F0000308F10083120B1DE22810308100FB
:100190000B110130AA02031CA90329082A04031D1C
:1001A000EB28A80A1E302802031DDD28FF30860038
:1001B000483085002F148B12EB280030A900323014
:1001C000AA00EB280C1CEB282C088F002D088E00B1
:1001D000803085060C1071088300F00E700E090047
:02400E00303F41
:00000001FF
